:100000000C9462000C948A000C948A000C948A0070
:100010000C948A000C948A000C948A000C948A0038
:100020000C948A000C948A000C948A000C948A0028
:100030000C948A000C948A000C948A000C948A0018
:100040000C9491030C948A000C9494010C948A00F3
:100050000C948A000C948A000C948A000C948A00F8
:100060000C948A000C948A000000000024002700F1
:100070002A0000000000250028002B0000000000DE
:1000800023002600290004040404040404040202DA
:100090000202020203030303030301020408102007
:1000A0004080010204081020010204081020000012
:1000B0000007000201000003040600000000000029
:1000C0000000190311241FBECFEFD8E0DEBFCDBF63
:1000D00011E0A0E0B1E0ECE3F9E002C005900D9280
:1000E000AA30B107D9F711E0AAE0B1E001C01D9232
:1000F000AC3AB107E1F710E0C4ECD0E004C02297BD
:10010000FE010E949804C23CD107C9F70E94530324
:100110000C949C040C94000080E991E00E94CA02B7
:10012000882329F180E991E00E94DE0290930B017F
:1001300080930A01009721F489E060E070E006C036
:100140008130910531F489E062E370E00E94CE00D5
:1001500008958230910529F48DE061E00E94470105
:100160000895039721F48DE060E00E94470108950F
:1001700080E991E040E855E260E070E00E94D10142
:100180008DE061E00E94270189E060E070E00E945C
:10019000CE008DE060E00E94470108951F93CF9349
:1001A000DF93182FEB0161E00E942701E12FF0E0BF
:1001B000E255FF4F8491833051F480918000806834
:1001C00080938000D0938900C09388003CC0843025
:1001D00051F480918000806280938000D0938B00E6
:1001E000C0938A0030C0813039F4209729F184B55A
:1001F000806884BDC7BD27C0823039F42097E1F004
:1002000084B5806284BDC8BD1EC0863041F4809133
:10021000B00080688093B000C093B30014C08730F2
:1002200041F48091B00080628093B000C093B4002C
:100230000AC0C038D1051CF4812F60E002C0812FB4
:1002400061E00E944701DF91CF911F910895282F0F
:1002500030E0C90186569F4FFC0194912A573F4FC9
:10026000F9018491882391F0E82FF0E0EE0FFF1F51
:10027000E859FF4FA591B491662329F48C9190958C
:1002800089238C9308958C91892B8C930895482F02
:1002900050E0CA0182559F4FFC012491CA01865645
:1002A0009F4FFC0194914A575F4FFA0134913323D9
:1002B000D1F1222331F1233021F4809180008F7716
:1002C00005C0243031F4809180008F7D80938000C0
:1002D00018C0213019F484B58F7704C0223021F47E
:1002E00084B58F7D84BD0DC0263021F48091B0008F
:1002F0008F7705C0273029F48091B0008F7D8093DF
:10030000B000E32FF0E0EE0FFF1FEE58FF4FA59176
:10031000B491662329F48C91909589238C93089548
:100320008C91892B8C9308951F920F920FB60F9288
:1003300011242F933F934F935F936F937F938F93EA
:100340009F93AF93BF93EF93FF934091C600E091CB
:100350008C01F0918D01CF01019660E870E00E9460
:1003600032049C0180918E0190918F0128173907EA
:1003700039F0E45FFE4F408330938D0120938C0170
:10038000FF91EF91BF91AF919F918F917F916F916D
:100390005F914F913F912F910F900FBE0F901F9043
:1003A00018955F926F927F928F929F92AF92BF92B9
:1003B000CF92DF92EF92FF920F931F93CF93DF9331
:1003C000EC013A014B01413482E458078FE06807A1
:1003D00080E078070CF07FC060E874E88EE190E080
:1003E000A40193010E9467042150304040405040D6
:1003F000CA01B90122E030E040E050E00E94670409
:1004000059016A01A60195012095309540955095B6
:1004100094E0220F331F441F551F9A95D1F760E0D7
:1004200074E284EF90E00E946704CA01B9012FEFE3
:1004300030E040E050E00E941304A40193010E94C8
:100440006704C90181509F4F181619061CF4522EDB
:100450005A9403C055245394521A60E079E08DE316
:1004600090E0A40193010E94670421503040404075
:100470005040CA01B90122E030E040E050E00E9463
:100480006704209530954095509583E0220F331FE7
:10049000441F551F8A95D1F760E074E284EF90E025
:1004A0000E946704CA01B9012FEF30E040E050E03C
:1004B0000E941304A40193010E946704C9018150A2
:1004C0009F4F181619061CF4822F815002C081E03C
:1004D000821B851500F5E885F98581E090E00A88A2
:1004E00002C0880F991F0A94E2F7808360E079E0E8
:1004F0008DE390E0A40193010E94670421503040F5
:1005000040405040CA01B90122E030E040E050E0F4
:100510000E94670404C0E885F98510829501EC818A
:10052000FD813083EE81FF812083EA85FB85208178
:1005300041E050E0CA010E8402C0880F991F0A945E
:10054000E2F7282B2083EA85FB852081CA010F84EE
:1005500002C0880F991F0A94E2F7282B2083EA85AE
:10056000FB858081088802C0440F551F0A94E2F77A
:10057000842B8083DF91CF911F910F91FF90EF909B
:10058000DF90CF90BF90AF909F908F907F906F90B3
:100590005F900895DC011296ED91FC911397E0585D
:1005A000FF4F8191919180589F4F20813181821B13
:1005B000930B60E870E00E9432040895CF93DF93BC
:1005C000DC011296ED91FC911397EF01CE57DF4FAE
:1005D00048815981E058FF4F80819181E058F04077
:1005E0008417950719F42FEF3FEF0CC0E40FF51FA8
:1005F0002081CA01019660E870E00E94320499836C
:10060000888330E0C901DF91CF910895FC01A08576
:10061000B18521898C9190E0022E02C09595879535
:100620000A94E2F780FFF6CF0484F585E02D60831D
:10063000089584E091E090939101809390018CE083
:1006400091E0909393018093920185EC90E09093D8
:1006500095018093940184EC90E0909397018093AE
:10066000960180EC90E0909399018093980181EC41
:1006700090E090939B0180939A0186EC90E0909398
:100680009D0180939C0184E080939E0183E0809390
:100690009F0187E08093A00185E08093A10181E024
:1006A0008093A20108950E94D9030E94B8000E947D
:1006B0008C00FDCF0F931F93CF93DF938C01EB0141
:1006C00009C02196D801ED91FC910190F081E02DB7
:1006D000C801099568816623A1F7DF91CF911F9129
:1006E0000F910895EF92FF920F931F93CF93DF9393
:1006F0008C017B01EA010CC0D7016D917D01D8010D
:10070000ED91FC910190F081E02DC80109952197B0
:10071000209791F7DF91CF911F910F91FF90EF906C
:1007200008951F920F920FB60F9211242F933F93AB
:100730008F939F93AF93BF938091A7019091A8014E
:10074000A091A901B091AA013091AB010196A11D20
:10075000B11D232F2D5F2D3720F02D570196A11DA0
:10076000B11D2093AB018093A7019093A801A093A2
:10077000A901B093AA018091A3019091A401A09135
:10078000A501B091A6010196A11DB11D8093A30101
:100790009093A401A093A501B093A601BF91AF913E
:1007A0009F918F913F912F910F900FBE0F901F90AF
:1007B0001895789484B5826084BD84B5816084BDC9
:1007C00085B5826085BD85B5816085BDEEE6F0E0CA
:1007D000808181608083E1E8F0E0808182608083B5
:1007E000808181608083E0E8F0E0808181608083A7
:1007F000E1EBF0E0808184608083E0EBF0E08081D9
:1008000081608083EAE7F0E080818460808380817A
:100810008260808380818160808380818068808322
:100820001092C1000895629FD001739FF001829FD2
:10083000E00DF11D649FE00DF11D929FF00D839F6F
:10084000F00D749FF00D659FF00D9927729FB00D0C
:10085000E11DF91F639FB00DE11DF91FBD01CF011F
:100860001124089597FB092E07260AD077FD04D09E
:1008700049D006D000201AF4709561957F4F0895F5
:10088000F6F7909581959F4F0895A1E21A2EAA1B25
:10089000BB1BFD010DC0AA1FBB1FEE1FFF1FA21730
:1008A000B307E407F50720F0A21BB30BE40BF50B2D
:1008B000661F771F881F991F1A9469F760957095B6
:1008C000809590959B01AC01BD01CF01089597FBE8
:1008D000092E05260ED057FD04D0D7DF0AD0001C04
:1008E00038F450954095309521953F4F4F4F5F4FCD
:1008F0000895F6F790958095709561957F4F8F4F8D
:100900009F4F0895AA1BBB1B51E107C0AA1FBB1F25
:10091000A617B70710F0A61BB70B881F991F5A958B
:10092000A9F780959095BC01CD010895EE0FFF1FAA
:0C0930000590F491E02D0994F894FFCF9D
:0A093C000000000006035A037203D6
:00000001FF
